:02000000462890
:080008008B13A000030EA10000
:10001000833081000514851405158515A603031981
:100020001D282608A700A70303192028A7030319E2
:100030002528A70303192A282F280530A6003428CD
:1000400022083B2086000510342823083B20860028
:100050008510342824083B20860005113428250803
:100060003B20860085113428210E8300A00E200E2F
:100070000B118B17090082071834DE3432345234E6
:10008000D43451341134DA3410345034FF30850014
:1000900086008316F030850000308600831204301D
:1000A000A2000330A3000230A4000130A5000530F7
:1000B000A6008316843081008330831281008B1662
:0400C0008B17612811
:02400E00F13F80
:00000001FF
